:020000040800F2
:10500000381A0020D550000875820008757A00080B
:105010000000000000000000000000000000000090
:10502000000000000000000000000000E18C00080B
:105030000000000000000000ED880008DD8D000881
:10504000E7500008E7500008E7500008E750000864
:10505000E7500008295B0008E7500008E750000807
:1050600000000000E7500008515A0008E75000080F
:10507000E7500008D17E000800000000E75000085B
:1050800000000000E75000080000000000000000E1
:10509000E750000800000000E7500008E750000853
:1050A000E7500008E7500008E75000085595000851
:1050B000E7500008E7500008000000000000000072
:1050C0000348854600F060FC0048004765A30008DF
:1050D000381A00200448804704480047FEE7FEE7EE
:1050E000FEE7FEE7FEE7FEE7798E0008C150000804
:1050F00030B50B46014600202022012409E00D4670
:10510000D5409D4205D31D469540491B25469540F7
:1051100040191546521E002DF1DC30BDF0B51FB40C
:105120000646002082B005464024019100901BE015
:10513000019922460F46304600F04EFB049A059B2B
:10514000801A994110D310461946224600F034FBCC
:10515000361A8F410197224601200021009F00F05E
:105160002BFB38184D4100902046641E0028DFDCE0
:10517000019B00982946324607B0F0BD03460B4319
:105180009B0703D009E008C9121F08C0042AFAD2FD
:1051900003E00B780370401C491C521EF9D2704783
:1051A000D2B201E00270401C491EFBD270470022BF
:1051B000F6E710B513460A4604461946FFF7F0FF16
:1051C000204610BD30B504460020034600E05B1CBD
:1051D000934203D2E05CCD5C401BF8D030BDF8B503
:1051E00002464A40D40F42004B0052085B089A42E4
:1051F00002D20246084611464A0023D0C30D4A0097
:10520000DDB2120EAD1A202D35DA49020126490A07
:10521000F6058A19002C00D0524220214F1B11465E
:10522000B9402A411018C20D9A4221D0002C17D043
:10523000012D08DCDA05801AD20F8019D207DBB203
:1052400000F0F6FAF8BDDA05801A012340001B06CB
:10525000C01880185A428018CA0F1043490007E04E
:105260004908C2071143DA05801A801940088018DE
:1052700000F0D6FAF8BD61000122511A001BF7E7D1
:105280000122D2075140AAE70122D2075040A6E7E7
:1052900070B502464A40D50F40004A00ED0740086D
:1052A0005208002814D0002A12D0C40DD30D410298
:1052B0000120C0055202490A520AE41A09181218BC
:1052C0007D34914201D3641C00E04900002C01DAD6
:1052D000002070BD0023914201D3891A0343400886
:1052E00049000028F7D100290AD0914202D10121BA
:1052F000C90705E0914201D2012101E00121C94322
:10530000E005C018401900F08BFA70BDF0B50746F3
:105310000846584087B0C00F049048000E46590018
:1053200040084908BC1A884105D2384631461E4615
:1053300017460B4602465800400810434CD0300D2B
:10534000039040055900400D490D0590401A029008
:10535000402872DA18030121000B09050843019067
:1053600004980092002805D00199524200208841FB
:1053700000920190029840210A1A0199009800F0C9
:105380001BFA05460C466B4607CB00F036FAC019EF
:105390007141039A0E0D0023D71756401A467A40E2
:1053A000164344D0049A002A2DD0029A012A039A67
:1053B00015DC1205C01A914101263605001C714109
:1053C000D20F059ED2070093019202962A462346E9
:1053D00000F074FA07B0F0BD38463146FAE716051A
:1053E000224A0F46B218C01AB74101210905001C14
:1053F0004F4100187F41114618187941E20F1043C0
:105400006D19644113E0E2076D0815436408C20793
:105410001443039A01261205C01A91413605001C57
:105420007141CE07400830434908C01851412A460F
:10543000234600F036FACDE7FFE70498012240004A
:10544000C117121A00238B4104983146C417381A29
:10545000A141EEE730B40124E407634030BC55E7D6
:1054600030B40124E407614030BC4FE70000E0FFA6
:10547000F0B51FB488B00B990998002448400999E9
:10548000C00F490049080991C0070B9900904900D5
:1054900049080B9109990898A64608431CD00B9916
:1054A0000A98084318D0099801244000420D48008A
:1054B000410D099824050003000B204309900B9827
:1054C0000003000B20430B9050181C494018002289
:1054D00001901446104605E0002001460DB0F0BDD5
:1054E000032801DA034600E003239C46C11A0AAEF2
:1054F0000AE05F0008ADED5B4F00F75B7D430027DE
:10550000AA187C41491C5B1E6145F2DD410004ABD9
:105510005A522104120C0A43240C401C0828DFDBD9
:10552000019802900099704601910090059B049AA1
:105530000799069800F0C2F9D0E700000DFCFFFFC4
:10554000F0B50C465C4085B0E40FE40703944C00D2
:1055500000266408590094464908024602962243F0
:1055600021D062460A431ED06200570D4A000E0346
:105570002303550D012402462C492405781B1B0BDF
:10558000360B401823432643614600901C46501AB0
:10559000B44103D30098401C009002E09218009898
:1055A0005B41002803DA0020014605B0F0BD002071
:1055B000012109050746864611E064461D46141B75
:1055C000B54106D36546521BB341744607430C43AD
:1055D000A646CD0740084908284392185B41054676
:1055E0000D43EAD11046184313D060461946504087
:1055F0007140084306D06046101AB34106D201221A
:10560000002306E000220123DB0702E00122D2434F
:105610005310009874460105381C6141029C039D9B
:105620000019694100F03DF9BFE70000FD030000EB
:10563000C217C10F504010B54018CA079623002169
:1056400000F0F6F810BD10B500229623114600F0C8
:10565000EFF810BD0EB5C217C10F5040CA07401871
:105660000021054B0293019200910A460B4600F07F
:1056700025F903B000BD0000330400000EB5054954
:105680000291002100910A460B46019100F016F9A3
:1056900003B000BD33040000410040020122400A73
:1056A000D205090E80187F2901DA0020704796295B
:1056B00003DC9622511AC8407047963988407047DB
:1056C00070B5CD0F4A0009030123090B1B051943CF
:1056D0000B4BED070024520D9A4201DA002070BDF9
:1056E000074B34339A4203DC9A1A00F075F802E053
:1056F0000449511888402C43F1D0404270BD00004D
:10570000FF030000CDFBFFFF4A0009030123090B43
:105710001B051943094B10B5520D9A4201DA0020BE
:1057200010BD064B34339A4203DC9A1A00F054F849
:1057300010BD03495118884010BD0000FF03000050
:10574000CDFBFFFFC20FD207400040080BD0C10DB8
:105750000723DB01C91840020905400A1143C208AA
:10576000400711437047002001467047CB0FDB070D
:10577000490010B5490802460A4307D00A0D07241C
:105780000903E401090B121B002A01DC002010BDF3
:10579000C900440F0C43C100E018D205801800F086
:1057A0003FF810BD0122D207002800DB101A0029A3
:1057B00000DB511A8142704710B5202A04DB0146F4
:1057C000203A9140002010BD914020239C1A0346AE
:1057D000E3401943904010BD10B5202A04DB084671
:1057E000203AD040002110BD0B46D340D0402024A9
:1057F000A21A91400843194610BD10B5202A06DBB5
:10580000CB170846203A1041C1170B4306E00B4660
:105810001341D0402024A21A91400843194610BDDC
:10582000002904DA401C490001D1400840007047BB
:1058300070B40024050C05D11024000402D1002905
:1058400021D01124050E01D100020834050F01D129
:105850000001241D850F01D18000A41C002801DB5C
:105860004000641C002908D020252E1B0D46F54061
:10587000A14000D001212943084301061B1B000A57
:10588000DB1D02D5002070BC7047DB05181880189E
:105890000029F8DA401C4900F5D170BC40084000EE
:1058A000704710B5002B08DA0024401C61419218A3
:1058B0005B411A4301D14008400010BDF0B51FB450
:1058C00082B005460C0003D0084603F001FF02E059
:1058D00003F0FEFE20300246009021462846FFF7E6
:1058E0006BFF049B059A04460F4618431143084377
:1058F00014D0184610431BD0009840210A1A1846AD
:105900000599FFF769FF05460E46009A0599049828
:10591000FFF752FF084305D0012004E02046394636
:1059200007B0F0BD0020C11705430E432C43374399
:1059300000990E986305401A7905E40A00220C4389
:10594000FD0A0A3002D500200146E9E701051019D9
:1059500069410C9C0D9D00196941FFF7A2FFDFE72B
:1059600010B5002904DB0124E40740428C412146A4
:10597000002B04DB1C460123DB075242A341994262
:1059800000D1904210BD0000064C0125064E05E0F6
:10599000E36807CC2B430C3C98471034B442F7D350
:1059A000FFF792FBC4A60008E4A6000838B5044639
:1059B000064805490068FFF79BFB604300E0401E76
:1059C00000900028FBD138BD40420F00EC000020C1
:1059D000F8B50446006881688907890F012902D15A
:1059E0000168C90722D18168114A1026114001259A
:1059F00000290ED18168294381600120FFF7D6FF7D
:105A000000F0A8FF07460CE000F0A4FFC01B0A2826
:105A100007D9606D30436065A06D2843A065012003
:105A2000F8BD20680068C043C007EDD10020F8BD74
:105A30001700008010B500231A4603E0845CE318C9
:105A40009BB2521C8A42F9D3D84380B210BD0000E9
:105A500010B5034800F03EFD024800F03BFD10BDCC
:105A6000D81500209015002030B5446C1C252C4022
:105A70000125A540046C6560046863608368102B91
:105A8000036803D099600068C26030BD9A60006806
:105A9000C16030BD1449012048720A4602205E32BE
:105AA000507203203C3A507204200E3A50720F4854
:105AB0000D4B0078087022310870203108770C49AE
:105AC0005A1C0878587149789971233318715971A3
:105AD000203318775977107551751A461E32107594
:105AE000517510765176704720110020BE000020BD
:105AF000D800002010B503F0CBF8202003F064F9A3
:105B0000012004F095F9002003F05EF9044804F048
:105B100033F8044804F0D6FA002004F00BFB10BD63
:105B2000A80000208380000070B505200121000737
:105B300000F000FF00240D4D002800D02C60022151
:105B40000B4800F0F7FE002808D10A482C600088B6
:105B50000A2148430849088003F00EFD012000F0A7
:105B600021FE022000F01EFE70BD0000E4000020B7
:105B700000040050CC000020D60000207047000038
:105B800010B5084900224A6107494B684C15234368
:105B90004B604B68082423434B60C009C00102607E
:105BA00010BD000020160020002002407FB5002517
:105BB0000C460646039500F0C5FDE009029003A9D6
:105BC00001960095684600F055FD002804D000F0CD
:105BD0008DFD002004B070BD00F088FD0120F9E7C4
:105BE00010B5002302E0C45CCC545B1C9342FAD392
:105BF00010BD000010B5214A00219069C30520485E
:105C000004D54169022319434161911593699B05AC
:105C100005D5436901242343436163021943936912
:105C20005B0505D54369082423434361E301194318
:105C300093691B0505D5436904242343436163022B
:105C4000194393699B0405D5436910242343436199
:105C50006302194393699B0304D5446920231C43C1
:105C6000446119439369DB0305D543694024234309
:105C70004361A0020143916110BD00000020024079
:105C80002016002070B5054600F064FE0646184C4C
:105C90000AE0681C08D0002D04D000F05BFE801BD9
:105CA000A84201D9032070BDA069C007F1D1A06945
:105CB000800701D50220A061A069C00511D4A069A8
:105CC00080050ED4A06940050BD4A069000508D456
:105CD000A069800405D4A069800302D4A069C00330
:105CE00003D5FFF787FF012070BD002070BD0000C5
:105CF00000200240F8B51746002605460C4600F085
:105D000021FD09E029460220226800F0FDFC002860
:105D100004D1241D2D1D361DBE42F3D300F0E6FC38
:105D2000BE4201D20020F8BD0120F8BD10B50849DF
:105D300002460020054B497905E044001C5B944273
:105D400003D0401CC0B28842F7D310BD48120020D7
:105D50004800002010B500F0F2FD10BD10B5094854
:105D600000F09AFF80B2FFF789FC074A074BFFF764
:105D70007FFB0022064BFFF7E3FBFFF7C5FC80B279
:105D800010BD000088140020F853E3A59B843E401A
:105D900000408F40F8B53F4C3D48217F0175617F41
:105DA00041753D490A78027649784176384905209F
:105DB000133148720A2004F075F9002004F08CF9C0
:105DC0003349002213310C2004F056FA00210C2034
:105DD00004F064FA022004F0B5F9304D00210F20E0
:105DE00004F0E0F82842E062F8D0E06A411C40D0BC
:105DF0002B4E2C4F40043ED58122D20100210F2092
:105E000004F00FFA0021102004F0CCF841062048DD
:105E1000490E0022633004F0FBF81D4D6335687AAB
:105E2000052825D102221C49681DFFF7CBF900285F
:105E30001ED1A87A607117480422691C4030FFF710
:105E40009DF9206C00F034F86083607929464200A7
:105E50000B3108465930FFF791F913483188808893
:105E6000FFF746F93888414310480180022020702E
:105E7000F8BD02F023FA608B31880546FFF738F948
:105E80003888414309486D1E01806583F8BD0000D4
:105E90008111002048000020D800002000D02724D5
:105EA000C8000020C6000020200D0020C4000020F3
:105EB00010B504460E4800F0EFFE0E49C006C00EB5
:105EC000098805E02246C240D2070FD0401CC0B26C
:105ED0008842F7D3012005E02246C240D20705D010
:105EE000401CC0B28842F7D3491EC8B210BD0000A2
:105EF00088140020C800002010B5084800F096FA69
:105F00000A21064800F032FA044800F01DF9800525
:105F100003D5024800F01AF980B210BD2C140020FD
:105F2000F8B52F4D00220121284600F00CFDFFF7A7
:105F3000E3FFFFF788FB2B4E3146FFF7A9F92A4C08
:105F40000122A0601146284600F0FDFC2749A06808
:105F5000002588423EDB2078254F002815D025708B
:105F6000FFF7CAFFFFF76FFB3146FFF791F9A0601B
:105F7000FFF7E8FB00223B46FFF76CFA00221D4BBF
:105F8000FFF776FAFFF7F2FB6060A068FFF7DAFB35
:105F900000223B46FFF75EFA174A184BFFF768FAF4
:105FA00006460F466068FFF7CDFB134A144B52427A
:105FB000FFF75EFA32463B46FFF7A8F9FFF7D6FB3C
:105FC00010496060884201DD616004E0FF21C9057D
:105FD000C84200D365606068FFF75EFBC0B2F8BDE1
:105FE0000004005000401B442400002000006040DA
:105FF00000000C4000E064403333333333B33040AF
:10600000CCCCEC3F0000C842F8B50546044640350C
:10601000287C0026012808D0012028742068816887
:106020008907890F01290ED101E00220F8BD01681E
:10603000C90708D0606D2021084360650126002053
:1060400028743046F8BD616DFF220132914302226F
:1060500011436165C1688907890F0091C16889088A
:106060008900C1602068816892071143816000F057
:1060700071FC07460EE000F06DFCC01B0A2809D930
:10608000606D022188431021084360650020287458
:106090000120F8BD206880680028ECDB2068C1681A
:1060A000009A1143C160606D80088000401C6065EB
:1060B000C5E70000F8B506460D464036317C01299B
:1060C0000DD00121317401688A68520709D5416DEC
:1060D000202211434165002030740120F8BD0220C8
:1060E000F8BD174B6A68D80547109A42154C8A6A62
:1060F0002B6812D05B035B0B1A438A622968490341
:1061000005D5A1680143A1600A20FFF74FFC28686C
:10611000800312D5A06838430EE05B035B0B9A4303
:106120008A622968490302D5A1688143A160286871
:10613000800302D5A068B843A06000203074F8BD89
:106140000110000000270140406D70470068006C9E
:106150007047000070B5040006D0606D264600252B
:106160004036002802D006E0012070BDA5653574D8
:10617000204600F0D3F8606DC00603D4216888681B
:10618000400705D5606D1021084360653574EBE765
:10619000606DFF22013290430222104360658868DF
:1061A0008207920F5B48012A02D10A68D2072BD1DD
:1061B000032362689B079A4205D05B429A4202D051
:1061C0005B009A4209D10A69920092080A6121682B
:1061D0000A6963681A430A610CE00A69920092082E
:1061E0000A6181680F22920491438160816862682C
:1061F000114381602168CA6818239A43CA602168E4
:10620000CA68A3681A43CA60816801225206914392
:1062100081608168A28E5206114381602068816886
:10622000C90004D4816801221207114381602068EB
:10623000C168394A1140C1602069E168022825D04F
:1062400000200143204620300278037B52035B008C
:106250001A431143226B1143A26992031143E2696D
:10626000D20311432268D3681943D160616A0A4698
:10627000FF3AC23A05D0A26A11432268D368194393
:10628000D16042780121012A02D00BE00420D8E736
:106290000078002823D0606D202210436065A06D37
:1062A0000843A065E06B012820681FD00169C90779
:1062B00003D0016949084900016120684169C908A2
:1062C000C900416120684169A26B11434161A56524
:1062D000606D80088000401C6065002070BD2068F3
:1062E000C26801231B041A43C260DBE70269FF2373
:1062F0009B009A43026120680269236CA66C1A43D2
:10630000636C33431A430261206802690A430261E5
:10631000D3E70000002701401902FEFF10B586B048
:10632000044614216846FEF742FF0E492068884261
:1063300016D10D48416B421511434163C16A0122D8
:106340001143C162C06A6946104005900220009066
:1063500003200190002002900520000700F02EFA93
:1063600006B010BD0024014000100240F8B50446FC
:106370004069254640350E4608280BD02068C06885
:10638000C00709D0606D2021084360650020287493
:106390000120F8BD082700E00C2700F0DBFA009090
:1063A00011E0701C0FD0002E05D000F0D3FA009938
:1063B000401AB04207D9606D04210843606500208F
:1063C00028740320F8BD206800683842E9D0606D69
:1063D00001214902084360652068C16809058A0FE8
:1063E0000C21002A1BD12022125D002A17D102683D
:1063F000120714D5826853070122002B08DB43687B
:106400008B434360606D130298431043606506E060
:10641000606D202318436065A06D1043A065A069DE
:10642000002801D1206801600020F8BD70B5044645
:10643000216800208968490721D425464035297CF8
:1064400001291CD001212974E169012904D02046C9
:10645000FFF7BEFA002811D1616D0A4A1140FF22F0
:106460000132114361650021A165297422681C2154
:10647000116021688A6804231A438A6070BD022073
:1064800070BD0000FEF1FFFF70B500240146203111
:106490004A79022A03D00421C163012418E002686A
:1064A00013680E25AB431360026813685B085B003A
:1064B0001360436C1C221340012215469D40036C5F
:1064C0005D604A7100220A71816B002900D0884703
:1064D000204670BDF0B4016C0D6801680C68466C14
:1064E0001C2304221E401746B7402F420ED06707D8
:1064F0000CD50C68A40602D40C6894430C60416C63
:1065000019408A40016C4A60016B1AE00227B740CB
:1065100002462F402032002F17D0A70715D50C6850
:10652000A40605D40C680A25AC430C600121517106
:10653000446C02211C40036CA14059600021117180
:10654000C16A002918D0F0BC08470827B7402F427D
:1065500012D0240710D50C680E25AC430C60446C97
:1065600001211C400B46A340046C6360C163517160
:1065700000211171416BE4E7F0BC704770B5040075
:106580003CD01F48256814212818FEF7B1FD800073
:1065900060641C482064022120462030024641717C
:1065A00029681948E3680140A068666918432369AF
:1065B00033431843A3691843E3691843236A184314
:1065C000084328600121A0688903884210D00D4843
:1065D0008030836A656C1C210D400F26AE40B343AA
:1065E0008362656C63680D40816AAB400B438362D4
:1065F0000020E06301215171107170BD012070BD58
:10660000F8FFFDBF000002400F80FFFFF8B5044611
:106610008C46203001790025012909D00126067118
:1066200041790027012905D0077102252846F8BDC8
:106630000220F8BD02214171E76320680168490822
:106640004900016061462046FFF70EFA206B0028E2
:106650002068016801D00E2205E004229143016008
:10666000206801680A2211430160206801683143F3
:106670000160DBE7F8B51A4E0546307C0F4601286D
:1066800007D0012030741748FFF7FCFA010002D050
:1066900021E00220F8BD0020C04338606C6814E09F
:1066A0002046FFF76DFA0F48FFF7ECFA01460E4857
:1066B000426808239A434260426843159A43426005
:1066C000002901D03C6006E08034A8686A68C001F7
:1066D0008018A042E4D8002030740846F8BD0000BD
:1066E0002016002050C300000020024005484168E9
:1066F00002221143416041680122114341600020A0
:106700007047000000200240F8B50C4C1646207C73
:106710000F46012808D0012020740948FFF7B2FA7B
:106720000025002802D006E00220F8BD65613E6029
:106730000348FFF7A7FA2574F8BD000020160020D3
:1067400050C3000011484168C9070BD0EFF3108116
:1067500072B60F4AC2600F4AC26081F31088416866
:10676000C9070ED1416889070DD5EFF3108172B6C4
:10677000094A0261094A026181F310884068800772
:1067800001D5012070470020704700000020024022
:10679000EFCDAB8905040302BFAE9D8C1615141313
:1067A0007047000010B504494A69024202D04861AE
:1067B000FFF7F6FF10BD000000040140F8B500230C
:1067C0000124A2E027469F403A4070D04D68022D38
:1067D00001D0122D14D1DD08AD002D1800952D6AC1
:1067E0005E07AC46F50E0F26AE46AE406546B54395
:1067F000AC460E697546AE4065462E43009D2E623E
:106800004D68012D05D0022D03D0112D01D0122D80
:1068100016D185680326AC465D00AE46AE4065469F
:10682000B543AC46CE687546AE4065462E4386609D
:1068300046680D79BE43ED06ED0F9D40354345603A
:1068400006685F000325BD40AE46AE430D79B446F1
:10685000AE07B60FBE4065462E430660C668754655
:10686000AE438D68BD403543C5604D68ED004BD5E6
:10687000294D6E6B26436E639E08284DB600751930
:10688000AC46AD689E07360F0F27B740BD430527BE
:106890003F07B84201D1002715E0214FB84201D18E
:1068A000012710E01F4FB84202D102270BE02BE076
:1068B0001D4FB84201D1032705E01C4FB84201D15A
:1068C000052700E00627B7402F436546AF60184D07
:1068D0002E684F689643FF0300D516432E606E68FE
:1068E0004F689643BF0300D516436E60AE684F688D
:1068F0009643FF0200D51643AE60EE684F6896439C
:10690000BF0200D51643EE605B1C0A681546DD40E9
:1069100000D057E7F8BD0000001002400000014021
:106920000004005000080050000C0050001C0050F3
:10693000000401400069084000D00120704742690E
:106940004A4042617047002A01D0816170478162EC
:10695000704700000148006870470000E800002010
:1069600002480168491C016070470000E8000020EF
:1069700010B50848002401684022114301602046F8
:1069800000F00AF8002801D0012401E000F0B0F97D
:10699000204610BD0020024070B5054609487D2103
:1069A0000024C9000068FEF7A3FB00F045FE0028A4
:1069B00001D0012404E000222946501E00F0B8F95D
:1069C000204670BDEC00002070477047F8B52C4C95
:1069D00001266078401C6070E670208B401C20838C
:1069E000208902F0BBF9274DE888FEF72CFE2649E6
:1069F000FEF74EFC254F3968FEF7F1FB38600221A7
:106A00002348FFF797FF002809D0002020621F4885
:106A10002049076820488F4212DD067012E0E8889E
:106A2000FEF711FE1849FEF733FC216AFEF7D7FB8B
:106A30001A4920628842EADB1A491948C860E6E729
:106A400000210170688F401EFEF7F2FD3946FEF707
:106A5000A9FE06D82079002803D01348C179314314
:106A6000C171688FFEF7EFFD08490968FEF79AFECD
:106A700004D22079002801D003F0F8FCF8BD000012
:106A8000BC000020200D002000007A44E40000201B
:106A900000040050000040404E0000200000A040D4
:106AA0000400FA0500ED00E094110020704770B575
:106AB00005000DD002202C462034A073284601F09A
:106AC0000FFA284600F0BEF80020A073607370BD76
:106AD000012070BD7047704710B50446006801681A
:106AE000C943C90708D18168C943C90704D1012135
:106AF00041602046FFF76AFF20680168C9438907A3
:106B000008D48168C943890704D402214160204622
:106B1000FFF75AFF20680168C943490708D4816814
:106B2000C943490704D404214160204600F0DEF83F
:106B300020680168C943090708D48168C943090767
:106B400004D4082141602046FFF7B0FF20680168A7
:106B5000C943C90608D48168C943C90604D41021B1
:106B600041602046FFF731FF20680168C94389066C
:106B700008D48168C943890604D420214160204695
:106B8000FFF7A9FF20680168C943490608D4816856
:106B9000C943490604D4402141602046FFF79AFFCB
:106BA00010BD0000F8B5040005D025462035A87BAF
:106BB000002802D006E00120F8BD002068732046BE
:106BC00000F052F80220A8732068C2688446636807
:106BD000012B04D00120A16AC005814201D11E20F1
:106BE000824315486169814201D01448024014482B
:106BF000A668024018463043676A266A3E4330431F
:106C0000A66A30431043012B03D00122D2059642DD
:106C100003D12369E2681A431043074A914205D021
:106C2000A2691143E2690243084610436146C86005
:106C30000120A8730020F8BDFFFF00003F1FFFFFE9
:106C4000F8F119FF10B500680549884207D10548D9
:106C5000816B4900490881630D2000F055F810BD93
:106C6000007C00400010024010B5006808498842CE
:106C70000CD10848816BC2041143816300220121B9
:106C80000D2000F055F80D2000F048F810BD000070
:106C9000007C0040001002400068C069704700009E
:106CA00070B50224034620339C730F4C2568E6041C
:106CB000354325600468E568B6123543E56005682C
:106CC000AE6801242643AE6005682E6926432E6116
:106CD0000568A96101684A610068016904221143DD
:106CE00001619C73002070BD0004014070470000EA
:106CF0000448416B012211434163816B020411433B
:106D00008163704700100240C106C90E012088400F
:106D1000014908607047000080E100E0C106C90E2B
:106D200001208840014908607047000000E100E050
:106D300010B501F0A1FA10BD02494A6882434A60C9
:106D4000704700000070004002480168821511433E
:106D5000016070470070004002494A6802434A607F
:106D6000704700000070004005480168022211438E
:106D700001600448016904221143016130BF70477A
:106D80000070004000ED00E00A4B1A689208920083
:106D900002431A600848036904221343036101296E
:106DA00006D040BF20BF20BF0169914301617047F9
:106DB00030BFF9E70070004000ED00E0F8B5044690
:106DC0000078544D800672D5524E0027403EB06B7D
:106DD000C00004D4B06BA9050843B06301274E4836
:106DE0000168C90511D40168821511430160FFF7DC
:106DF000B1FD009005E0FFF7ADFD0099401A642851
:106E000037D845480068C005F5D532680321090523
:106E100060680A400140914208D08103890F03292C
:106E200004D13168890301D50120F8BD2A69032105
:106E300009040A4022D0084090421FD020788006E2
:106E40001CD528692A6988430121C9040A432A619B
:106E50002A698A432A612861C0050FD5FFF77AFDA8
:106E6000009008E0FFF776FD0099411A2B48814217
:106E700001D90320F8BD28698005F3D5616888032E
:106E8000800F032805D132680005824301400A4380
:106E900032602869032261681204114008432861A6
:106EA000002F04D0B16B012000078143B16320782B
:106EB000C00705D0E868A168800880000843E86042
:106EC0002078800705D5E8680C218843E1680843ED
:106ED000E8602078400706D5E868032189028843E6
:106EE00021690843E8602078000706D5E868032197
:106EF0000903884361690843E8602078000606D5E5
:106F0000E868032189048843A1690843E8600020F8
:106F1000F8BD0000401002400070004088130000DF
:106F2000F8B50E4605007DD053480068C007C00F75
:106F3000B0420AD250480168490849003143016013
:106F40000068C007C00FB04271D128784B4C800751
:106F500005D5E068F0218843A9680843E0602878F7
:106F6000C00752D06868022817D0032818D02168BB
:106F7000012818D08905002959DAE16889088900B3
:106F80000143E160FFF7E6FC69680746022912D079
:106F900003291CD0012926D033E021688903EAE7C0
:106FA00021688901E7E74907E5E7FFF7D3FCC11B43
:106FB0003348814223D8E0680007800F0228F4D1CB
:106FC00023E0FFF7C7FCC11B2D48814217D8E068BA
:106FD0000007800F0328F4D117E0FFF7BBFCC11BAB
:106FE000274881420BD8E0680007800F0128F4D1C0
:106FF0000BE0FFF7AFFCC11B2148814201D9032000
:10700000F8BDE0680007800FF3D11B480168C9078D
:10701000C90FB1420DD901684908490031430160E7
:10702000006800E003E0C007C00FB04201D00120BB
:10703000F8BD2878400706D5E06807210902884393
:10704000E9680843E0602878000707D5E068072171
:10705000C90288432969C9000843E06000F036F896
:10706000E168084A0906090F515CC84006490860F2
:107070000020FFF791FCF8BD002002400010024004
:1070800088130000A2A60008EC000020044805496F
:107090000068C968044A4905490F515CC8407047F7
:1070A000EC00002000100240BBA60008044805497F
:1070B0000068C968044A8904490F515CC840704798
:1070C000EC00002000100240BBA6000810B5184AD2
:1070D000D1680C20084004280BD0082810D00C28B8
:1070E00010D050680004410F0120C003491C8840A3
:1070F00010BD1068C00601D50E4810BD0E4810BD69
:107100000E4810BD88020E4B000F185C0902D368B0
:10711000890F491CDB0301D5084A05E01268D20635
:1071200001D5044A00E0044A5043FDF7E1FF10BDD9
:107130000010024000093D000024F40000127A0013
:10714000B2A60008FEB505007ED0FE4CE7680C2014
:10715000E66807400120000406402878C00747D0B1
:10716000082F05D00C2F0AD101200004864206D139
:10717000206880033CD568680028E5D038E001200D
:1071800069680004814203D121680143216011E054
:10719000052301221B0492049942216802D1114364
:1071A0002160F1E78143216021680140009120685E
:1071B00090432060686800280DD0FFF7CBFB00905B
:1071C00005E0FFF7C7FB0099401A64287AD82068C9
:1071D0008003F6D50CE0FFF7BDFB009005E0FFF75C
:1071E000B9FB0099401A6428F0D820688003F6D4CF
:1071F0002878800755D50923E868042F0DD00C2F77
:1072000001D1002E09D000283BD0216899430143C9
:107210002160FFF79FFB064627E02168490701D55B
:10722000002891D061681F22120291432A6912023C
:10723000114361602168994301432160FFF746FFD4
:10724000E16809060A0F00E079E1BF49895CC8409E
:10725000BE4908600020FFF79FFB002872D120E0A4
:10726000FFF778FB801B0228B0D820684007F7D5CD
:1072700060681F2109028843296909020843606088
:107280000FE02068400840002060FFF763FB0646DF
:1072900004E0FFF75FFB801B022897D820684007B7
:1072A000F7D42878C0065FD5002F0CD0A869002835
:1072B00049D02068FF21013108432060FFF74AFBD5
:1072C00006462DE0C0E02068800502D5A8690028A8
:1072D000A7D06068072149038843296A0843606092
:1072E0006068297F0002000A090608436060286A76
:1072F000410B0120C003491C8840E16809060A0FC0
:107300009149895CC840914908600020FFF744FB1F
:10731000002817D128E0FFF71DFB801B0228A3D807
:1073200020688005F7D56068072149038843296AEA
:10733000084360606068297F0002000A090608436C
:10734000606011E0E1E02168FF20013081432160AD
:10735000FFF700FB064604E0FFF7FCFA801B02285B
:1073600072D820688005F7D42878794E000724D594
:1073700068690028306910D0012108433061FFF7A7
:10738000E9FA009005E0FFF7E5FA0099401A0228B3
:107390005AD830698007F6D50FE0400840003061C8
:1073A000FFF7D8FA009005E0FFF7D4FA0099401AE9
:1073B000022849D830698007F6D42878400765D577
:1073C00000200290A06BC00006D4A06B0121090729
:1073D0000843A063012002905E480168C90511D4EA
:1073E0000168821511430160FFF7B4FA009005E0CF
:1073F000FFF7B0FA0099401A642825D8554800686C
:10740000C005F5D5FF20AA680130824203D1316959
:107410000143316111E001218902002A07D00523CF
:107420001B029A4203D132690A433261EFE73269A3
:1074300082433261306988433061A86800280FD0E8
:10744000FFF788FA009007E05EE0FFF783FA009903
:10745000411A4148814257D830698005F5D50DE081
:10746000FFF778FA009006E0FFF774FA0099411AE6
:107470003948814248D830698005F5D402980028FF
:1074800004D0A06B012109078843A063686A002823
:1074900064D00C2F3ED0012636060228206805D085
:1074A000B0432060FFF756FA05462FE0B043206056
:1074B000FFF750FA074604E0FFF74CFAC01B02281A
:1074C00022D820688001F7D4E96AA86AE2680843F4
:1074D000296BFD231B049A4311430843E060206895
:1074E00030432060FFF736FA054604E0FFF732FA32
:1074F000401B022808D820688001F7D52EE0FFF74E
:1075000029FA401B022801D90320FEBD2068800112
:10751000F5D423E00128F8D0E06801210904AA6A23
:10752000014091420BD10F218904EA6A0140914246
:1075300005D1032189050840296B88420ED001201E
:10754000FEBD000000100240A2A60008EC000020D2
:107550004010024000700040881300000020EFE758
:1075600070B5040007D0002625464035A662687C29
:10757000002802D005E0012070BD2E74204600F0E6
:107580002FF802206874206801684022914301604E
:10759000A168606822690843E16811430843616992
:1075A00001220843A169520211400843E1690843DE
:1075B000216A0843A16A084321680860A069042180
:1075C000000C0840616A0843216848602068C1696E
:1075D00092009143C161666501206874002070BD0E
:1075E00010B586B0044614216846FDF7E0FD104949
:1075F0002068884219D10F48416B821411434163BE
:10760000C16A01221143C162C06A00211040059085
:10761000E020009002200190032003900291049149
:10762000052069460007FFF7C9F806B010BD000045
:107630000030014000100240094910B5401E884248
:1076400001D9012010BD074C60610321081F00F023
:1076500013FE0020A06107202061002010BD000063
:10766000FFFFFF0000E000E070477047F8B50268D8
:107670000446D0691168936805072D0F5BD0DD07BC
:10768000ED0FFF2621360E402E4367D0C60706D0E9
:10769000CE0504D501261662E26F3243E267870702
:1076A00002220426002F06DADF0704D027683A6298
:1076B000E76F3743E767470706D5DB0704D0236842
:1076C0001E62E36F1343E367020709D520220A40D5
:1076D0002A4305D0236808221A62E36F1343E36745
:1076E000E26F002A2FD0800606D5880604D5216EC9
:1076F000002901D020468847E06F21688968490643
:1077000001D4000724D5204601F094FD206881684B
:10771000490619D58168402291438160E06E0028B6
:1077200012D020498163E06EFEF7AEFE00280AD039
:10773000E06E816B06E0850610D58D060ED5216EB4
:107740001CE020468847F8BD2046FFF78EFFF8BDB5
:107750002046FFF78AFF0020E067F8BDC50208D584
:107760005B0206D50120000510622046FFF77CFF72
:10777000F8BD030605D50B0603D5616E0029E0D1DF
:10778000F8BD4006FCD54806FAD5136820464021CE
:107790008B431360202161670021616600F069F965
:1077A000F8BD00009191000810B5040003D0606F8F
:1077B000002802D007E0012010BD002170200155F3
:1077C000204600F027F824206067206801684908F7
:1077D00049000160204601F077FD0128ECD0606A85
:1077E000002802D0204601F0B5FB2068416809223C
:1077F000D20291434160206881682A2291438160CE
:1078000020680168012211430160204601F008FC54
:1078100010BD0000F0B587B0064614216846FDF79C
:10782000C6FC2C493068884251D12B48416B01225B
:10783000920311434163C16A01221143C162C06ACC
:1078400000251040059003204002009002200327ED
:1078500001A9A1C104200490052069460007FEF794
:10786000ADFF1F4C1D48A560E56081C48027E56021
:10787000A7602020256160610002A0611848083CD3
:10788000FEF77CFE002801D0FEF778F9F466A662C8
:10789000144C1248214614382060032060601020E8
:1078A0000831A1C16561A561E56120462562FEF749
:1078B00065FE002801D0FEF761F9B46600220121BF
:1078C0001B20A662FFF734FA1B20FFF727FA07B048
:1078D000F0BD0000003801400010024030000240BE
:1078E00090150020D8150020F8B50446806F202898
:1078F0004DD100290BD0002A09D00123A0681B0319
:10790000984206D12069002803D1C80701D0012080
:10791000F8BD25466035287C012838D00120287420
:107920005820616502530026E6672220A067E06EBA
:10793000002819D01749C162E16E17480863E16E4B
:1079400016484863E06E13468663676D21683A46C1
:107950002431E06EFEF75AFE002805D01020E067C3
:107960002E7420206067D2E72E7420680168FF2201
:107970000132114301602068816801221143816056
:10798000206881684022114381600020F8BD0220F8
:10799000F8BD0000ED9100082B920008A5910008A9
:1079A00070477047FFB50446406F83B017460D46D9
:1079B00020285CD1002D0AD0002F08D0A168C0017A
:1079C000814207D12069002804D1E80702D00120B4
:1079D00007B0F0BD204660300290007C012846D000
:1079E0000298012101740020E06721206067FEF702
:1079F000B1FF264640360190378277820120A16888
:107A00000003814202D12069002802D02F460025C0
:107A100011E000270FE000228021204601F068FDE0
:107A2000002815D1002F15D02168387888627F1C76
:107A3000708A401E7082708A019B00280698009010
:107A4000E9D100224021204601F052FD002808D053
:107A50000320BDE728882168C005C00D8862AD1CE1
:107A6000E6E720206067029900200874B0E7022052
:107A7000AEE77047FEE710B5052424070022042175
:107A80002046FEF760FF002208212046FEF75BFF3C
:107A90000A2002F02AF8012204212046FEF753FFB3
:107AA0000A2002F022F8002204212046FEF74BFFB4
:107AB00010BD10B505242407002204212046FEF73E
:107AC00042FF012208212046FEF73DFF0A2002F076
:107AD0000CF8012204212046FEF735FF0A2002F0AF
:107AE00004F8002204212046FEF72DFF10BDF8B552
:107AF0000024052607462546360700220421304685
:107B0000FEF721FF0A2001F0F0FF01220421304698
:107B1000FEF719FF6006040E08213046FEF70AFF43
:107B2000002801D0641CE4B2052001F0DEFF6D1CCA
:107B3000EDB2082DE1D3002F03D0FFF79CFF2046C4
:107B4000F8BDFFF7B6FFFAE770B50526054636071C
:107B5000002204213046FEF7F6FE0024E80901D099
:107B6000012200E0002208213046FEF7ECFE680604
:107B7000050E0A2001F0B9FF012204213046FEF76C
:107B8000E2FE0A2001F0B1FF002204213046FEF798
:107B9000DAFE0A2001F0A9FF641CE4B2082CDDD350
:107BA00070BD10B505242407012208212046FEF7E8
:107BB000CAFE012204212046FEF7C5FE002208214C
:107BC0002046FEF7C0FE0A2001F08FFF00220421AC
:107BD0002046FEF7B8FE10BD10B50524240700228C
:107BE00004212046FEF7AFFE002208212046FEF7C2
:107BF000AAFE0A2001F079FF012204212046FEF7A7
:107C0000A2FE012208212046FEF79DFE0A2001F077
:107C10006CFF10BD70B505252D0700240122082139
:107C20002846FEF790FE062001F05FFF01220421A6
:107C30002846FEF788FE062001F057FF07E0641C87
:107C4000E4B2FA2C03D9FFF7C7FF012070BD082169
:107C50002846FEF76FFE0028F1D1002204212846B5
:107C6000FEF771FE002070BDF8B501F009FA01F0D1
:107C700043FA4C480068C0694B4E4C4F800700D512
:107C8000FE60FEF76BF84A4C0246608849490028BE
:107C900003D0401E6080012008700878012189020D
:107CA000454D00281CD0012804D0022804D0032808
:107CB00006D115E0212A13D200222846FEF743FE02
:107CC0000121C9023C48FEF735FE3C490025002849
:107CD00028D03B48056008468079002802D006E09D
:107CE0000122EAE735490120887101F045FC33485B
:107CF0000078632806D9002208212F48FEF723FECA
:107D0000012205E0012208212B48FEF71CFE00227B
:107D100001210520C9030007FEF715FEA08C0128EC
:107D200003D01CE08D710022EDE7264869460880EB
:107D300072B680212448FDF739FF002804D00222C2
:107D400069462148FDF7D6FF62B620A001F0B0FCDD
:107D5000A58402F027FC642001F0C0FEFE60608C68
:107D6000012809D1124865844038058002F01AFCC8
:107D7000642001F0B3FEFE60208C012806D125842A
:107D800002F010FC642001F0A9FEFE600848134ACE
:107D900040380188914202D1C088002800D1FE609D
:107DA000F8BD0000101500200400FA0500ED00E009
:107DB000600D00205A00002000040050BC0000208C
:107DC000E4000020AAAA0000384A0008BDF8C8EB69
:107DD000C9FDBCB6C4A3CABD0D0A0000AA55000067
:107DE00008B53721202000F06EF80321212000F093
:107DF0006AF84021222000F066F80821232000F0D4
:107E000062F8AA21302000F05EF80A4802210187BA
:107E1000322000F058F80121332000F054F85F219F
:107E2000202000F050F8684600F006F80A2001F023
:107E30005CFE08BD200D002010B501460F2000F0AB
:107E400021F8002800D0012010BD10B50446FFF72E
:107E5000A8FE3220FFF778FEFFF7DCFEE0B2FFF766
:107E600073FEFFF7D7FEFFF79CFE3320FFF76CFE93
:107E7000FFF7D0FE0020FFF73AFE0446FFF7ACFE06
:107E8000204610BD10B50C46FFF7DFFF2070012023
:107E900010BD70B50D460446FFF783FE3220FFF794
:107EA00053FEFFF7B7FEE0B2FFF74EFEFFF7B2FE5C
:107EB0002846FFF749FEFFF7ADFEFFF78DFE0A20CB
:107EC00001F013FE70BD10B5FFF7E3FF012010BDF8
:107ED00010B50248FEF700FE10BD00008814002017
:107EE000FEB50446002572B60068394A831804D1ED
:107EF0003849CD68032189040D4081680191C1682A
:107F0000009141698669002B08D132484038836A64
:107F1000C7043B438362836ABB43836208463043A2
:107F200048D02B482368C34205D12A48C36803229E
:107F300092049343C360002917D02068026901238B
:107F40001A43026120684161FEF704FD0746FEF70F
:107F500001FD2168C01B0968090703D47D21C90000
:107F60008842F4D9216808204860002E17D0206884
:107F7000016901221143016120688661FEF7EAFC74
:107F80007D270646FF00FEF7E5FC2168801B096897
:107F9000C90601D4B842F6D92168102048600C48BF
:107FA0002168C14206D10B48C16803229204914363
:107FB0002943C160206801694908490001612168BD
:107FC0000198886021680098C86062B6FEBD000014
:107FD0000084FFBF401002401CB5002116480091EC
:107FE000144A01910260C163120542608160072258
:107FF0008263012202610246C16020321170FF23B8
:108000005170C23343628162117301638161042242
:1080100041634261C161FEF79DF8084800908013FA
:10802000019069460448FEF745F800210248FDF733
:10803000EBFF1CBD002401402C14002002000004B2
:1080400008B50848016B012211430163006B01214F
:108050001040009000220A20FEF76AFE0A20FEF778
:108060005DFE08BD00100240F0B587B014216846DF
:10807000FDF79DF84C48C26A04210A43C262C26AF5
:108080000A400592C16A80273943C162C16A3940FA
:108090000591C16A01252943C162C16A2940059140
:1080A000C16A02263143C162C06A2A463040059047
:1080B00005201C210007FEF746FC01223B493C48F5
:1080C000FEF741FC00223B493948FEF73CFC912178
:1080D0000520002209020007FEF735FC3648019012
:1080E000002405206946009502940007FEF766FB10
:1080F0000320019005206946009602940007FEF7D0
:108100005DFB0C20009011200190032003900520BE
:10811000029469460007FEF751FB102000900520ED
:1081200069460396019502940007FEF747FB11206C
:10813000019002946946009503941D48FEF73EFBAA
:108140001E4801906946009602951948FEF736FBD5
:108150001B48009002946946019503941448FEF769
:108160002DFBE8026A4651C269461148FEF726FB1C
:108170009120000200900520029469460195039425
:108180000007FEF71BFB694609480097029501941A
:10819000FEF714FB002201210520FEF7C9FD052092
:1081A000FEF7BCFD07B0F0BD001002400106000064
:1081B00000040050083000000000111000002110E1
:1081C0000836000010B50F4C0D482060FF20053028
:1081D00060600020A060E06020616061E0610121DA
:1081E000206249026062A161A0620720E06220462D
:1081F000FFF7B6F92068016840221143016010BD05
:1082000000300140B814002000B585B01421684644
:10821000FCF7CDFF164815490160E1214902416094
:1082200000218160C160016181610C22C1614261F4
:108230000162302141620121090381634900C16368
:10824000FFF7B2FA01208002009002200190012085
:108250000290032003900420049005206946000743
:10826000FEF7ACFA01F082F905B000BD003801401C
:1082700010150020704700008307FF22DB0E9A4094
:108280008907090E994000280BDA0007000F08380B
:10829000830808489B001818C36993430B43C361C4
:1082A0007047830804489B001B18186890430843D4
:1082B0001860704700ED00E000E400E0BFF34F8F6E
:1082C00004490348C860BFF34F8F00BFFDE70000BB
:1082D0000400FA0500ED00E0F0B585B00A2001F0D9
:1082E000E1FE002001F0F8FEF84D0024AC70A87B00
:1082F0000C2801D30B20A87301220520510200078E
:10830000FEF721FBEC70F248AC74F24E007830714D
:108310000221F148FEF70EFB002860D00020A97969
:10832000EC4E49000843F071A86AF070401CA86246
:1083300068793146B0724200B4310846A938FCF77A
:108340001DFF0620707230461338297F0175697F42
:10835000417568790022400031460D3001F08CFFF4
:108360006879002140000D3001F098FF022001F0F3
:10837000E9FE0024F4712C74AC7201202873EC72B5
:10838000D648FEF789FC28840646EC706879FDF72C
:1083900075F9D34AD34BFDF76BF801F03BFB012392
:1083A00000229B07FCF7B2FFFDF7AEF90006C10CF7
:1083B000881980B20121C9036884884201D3401A18
:1083C0006884C94868632879401C2871C348FEF74F
:1083D00063FCE883BF48C54C4E30029071E1012038
:1083E0009DE7BE48FEF758FCE883C14F0AE0BB4852
:1083F000FEF752FC80B2E883698C884202D30919E7
:10840000884206D300210F2001F0CCFD3842E862FB
:10841000EDD0E86A411C20D02E4640047ED5812252
:10842000D20100210F2001F0FCFE002001F054FEDB
:10843000002001F006FE0021102001F0B3FD4106EE
:10844000A448490E00225030019101F0E1FDA148FD
:108450005030417A0729C1D101E0FFF72FFF9D4835
:108460000222A4495530FCF7ADFE0028B6D101F038
:1084700066FFF164B06401F04FFF71653065F0781C
:108480009449401CF0704D310A7968460270497970
:1084900041700088B18B88427ED10298964F008A45
:1084A00038808C484C30808A30838C48FEF7F4FB4F
:1084B000F083308B9149FF30C33080B230838842E3
:1084C0000CD949424018308338888C49401C80B20E
:1084D0000B313880884201D30020388002987B4AD3
:1084E00081891186C0895086326B7263794A503215
:1084F000D27C13071B0F032B00D0B3741209F27444
:10850000002333710123B372704B002A9986D886F9
:1085100015D0704802227749553000E0C5E0FCF7DD
:1085200051FE00280BD101206A493074C8710198AE
:1085300064311638C2B272747148FCF71FFE012014
:10854000F07264496148042251314030FCF716FE54
:108550006048736D1630326D01F0C6FE3F887D2095
:10856000C000318B78434018B063049065480178AF
:10857000F17365480191C088FDF765F800903846B1
:10858000FDF761F80099FCF783FE7F21C905FCF730
:1085900026FEFDF781F800E02BE05A4980B2088002
:1085A0000199491E884201D10120F072B78414203C
:1085B000305EFDF74FF801910090F08BFDF75EF80B
:1085C000524A534BFCF754FF074603910498FDF7BA
:1085D00041F83A46039BFCF73DFF019B009AFCF7EC
:1085E00095FEFDF76DF8F0634A48008800F0B6FB91
:1085F00067E0FDF79BFB0746414803210C38C15556
:108600000298324982890A86C08948863C4AB80065
:108610009C3A316B11502F49736D40181A30326DEE
:1086200001F062FE70797F1C87424AD101F0D8FBCD
:10863000FF23296D5B04686D0022C91850410006B4
:108640000C0A044360084000010E0002E965A865B9
:108650002048EB6C0A30AA6C01F046FE1D48EB6D19
:108660001230AA6D01F040FE1A4808214172687963
:108670000022800017491C3001F0FEFD68790021BE
:1086800080001C3001F00AFE204601F004FD0120AC
:1086900001F058FD0006000E287240D100210F2085
:1086A00001F080FC0006F9D539E03A4600210F20A0
:1086B00001F0B7FDF0787179884202D0002001F016
:1086C000C0FCE98B688C814226D28AE648000020F3
:1086D000BC000020941100200004005088140020E9
:1086E000B81E85EB51B8CE3FA0860100983A000035
:1086F00000D02724D8000020E0000020E70300007D
:1087000014130020D4000020200D0020F853E3A50E
:108710009B843E40C400002000198142D5D86D4A98
:1087200000210F2001F07DFD6B4800240078002817
:1087300003D16A48008800F011FB002768493846D9
:108740008F734A79039221E0634B195C00291BD097
:10875000634DA300AE7B9C46761CAE735E4D6600F7
:10876000303DE9505C4B4500C03B5D5B18339D5389
:1087700085001833584E5D596346603EF550641CC1
:10878000554B491EE4B21954401CC0B29042DBD391
:108790005348C178032901D2817B8173504900225B
:1087A000887B4873401E35E000212FE04A4D8B0046
:1087B000603DEC585E1901967668B446644523DD49
:1087C00000944C00483D2D5B9600AE46424D303D36
:1087D000AD59414E02956546603EF5503546483DDF
:1087E0006519AC466D88483E3553344678341E19B9
:1087F000394D7468303DEC50019C009B63607546B8
:1088000063465D80029D7560491CC9B28142CDDB23
:10881000521CD2B28242C7DB2F486038026830480F
:10882000416B32398A421ADA2B49303909680029FA
:1088300015D0C179491CCAB2C271032A05D9264A8A
:10884000A83A12888283012202700179032900D993
:108850000770214B00210478C03B039A08E0C771E0
:10886000F3E74D005D5B002D00D10124491CC9B226
:108870009142F6D3184B00211A4A0470903B8C00A9
:10888000491CC9B21A510C29F9D3007C002806D022
:1088900011490C3108784B788A7802280ED00D4A9D
:1088A000002180320F2001F0BCFC012105200022B4
:1088B00049020007FEF747F805B0F0BD0A48C91C99
:1088C000C018FCF75BFC01F06DFE642001F006F9B6
:1088D000C3E5000000D0272408130020C4000020B6
:1088E00048000020FFFF0100200D0020704700001D
:1088F000F0B589B0934800900020C0430590002651
:108900000A2001F0CFFB002001F0E6FB00208E4C96
:108910000546A0708D4F8E4806908D480022C238C3
:1089200085730146142001F0A7FC0021142001F0FA
:10893000B5FC022001F006FC00210F2001F032FB03
:108940003842E062F8D0E06A411C18D040047DD57E
:108950008122D20100210F2001F063FC00211020B0
:1089600001F020FB41067A48490E0022801C01F0EC
:108970004FFB7748801C417A022902D0C1E0FFF703
:108980009DFC734802227349C01DFCF71BFC0028A4
:10899000F4D101F0D4FCE164A06401F0BDFC616598
:1089A0002065002E22D106996B48098A018068480B
:1089B0000126801E808A20836848FEF76DF9E083D7
:1089C000208B6749FF30C33080B2208388420DD9A5
:1089D00049424018604920830888614A401C80B29F
:1089E0000B320880904201D3002008800698694627
:1089F00082898A80C089C88055490422C91C0846DA
:108A0000A238FCF7BBFBFF22216D5204606D0023EE
:108A1000891858410006090A01430846029101F0ED
:108A20003AFB029948084000010E0002E165A0658A
:108A30004748E36C9638A26C01F056FC4448636DDD
:108A40009238226D01F050FC414800E05BE08E3826
:108A5000E36DA26D01F048FC3D490022A0393C20A5
:108A600001F00AFC00213C2001F018FC012001F07B
:108A700069FB2072A0780121401CA0700520C90369
:108A80000007FDF767F9206CFDF712FA02903548F0
:108A900001880298FCF72CFB33480088414388B2D8
:108AA000324908800299491E618300F057F9019903
:108AB000009881420DDA00290BD025490422C91CF7
:108AC00005A8FCF75BFB012020700520607201986F
:108AD0000090207A002805D100210F2001F062FAD1
:108AE0000006F9D5802200210F2001F09AFB00201A
:108AF0006D1CEDB26070032D00D20EE7002E08D081
:108B00001BE00120F4E71A4A00210F2001F089FB45
:108B1000F7E7608B401E0004000C608303D011490E
:108B20000988884202D90F48018861830E49608B09
:108B30000988401E48430D4908800598A08309B064
:108B4000F0BD00003F420F004800002000D0272465
:108B5000E2110020D8000020E0000020881400204E
:108B6000E7030000C8000020C6000020C400002069
:108B700000902724F8B52D492B48086001F0B2FC7D
:108B80002C4D2B486880E888002801D16420E880BB
:108B900029480178432901D943210170E98E0170E8
:108BA000264CE88F2071A88F6071A87AA070AE88DB
:108BB0000521E6616181EF883846FCF799FAA081CA
:108BC00001463046FCF794FA8800081886B27D20EA
:108BD000C00026817043FCF751FD194A194BFCF780
:108BE000AFFCFCF791FDE0817D2066823946C00034
:108BF000FCF77EFA2082E08201202083FDF7AEF8A8
:108C0000A082E28910491148FEF74AF810A0E169F4
:108C100000F04EFDE98812A000F04AFD298915A058
:108C200000F046FDF8BD0000A595000844000020B6
:108C300002020000200D002000000020BC000020E7
:108C4000F853E3A59B843E40FF7F0000881400207A
:108C5000B1EAC7A949443A202564202E0D0A000034
:108C6000CDA8D1B6BCE4B8F43A202564206D732EAB
:108C70000D0A0000B5A5B4CECDA8D1B6BBF9D5BEBE
:108C8000CAFDC1BF3A202564B8F62E0D0A000000C7
:108C900070B586B014216846FCF789FA01250F4E9D
:108CA000ED03002229463046FDF74DFE0120002449
:108CB000019002946946009503943046FDF77EFDCD
:108CC0000320019002946946009503943046FDF715
:108CD00075FD022000F002FF06B070BD00040050D8
:108CE00070470000F8B5044600206A461080194D10
:108CF00055222A70AA226A700322AA70661DEE709D
:108D00002A716971144A49008918AC712246E81D1C
:108D1000FCF734FA002007E029186A46897812889F
:108D200089186A461180401CB042F5DB611DA81C01
:108D3000FCF780FE01466846018029190078C87159
:108D400068464078087221460931024800F08AFAE4
:108D5000F8BD0000C8130020200D002010B51349F5
:108D60000A8BCB8A9A4201D3D21A0A83104A098B02
:108D7000D2884A437D211018C90048430D4909682B
:108D8000401AFCF767FC0C4A0C4BFCF7D9FBFCF7CC
:108D900097FC0B49884201DD4A428018002800DA1E
:108DA000401808490968486110BD0000BC00002057
:108DB000200D002084000020F853E3A59B843E4052
:108DC000FF7F000088140020034A1168382389B20D
:108DD00099430143116070470030014010B5FDF721
:108DE000BFFD10BD10B59AB034216846FCF7DFF91D
:108DF00014210DA8FCF7DBF91C2112A8FCF7D7F908
:108E00001B4801680324E402A143C21489180160CD
:108E1000FDF79AFF17480169A14301610620009000
:108E2000FF200130029001200390102004900220C6
:108E3000099040040B90000100240C900A946846AD
:108E4000FEF780F90F200D9003200E900F941094E0
:108E5000012111940DA8FEF763F8812012900320E0
:108E600080041890149412A8FDF7A8FF1AB010BD42
:108E70000070004040100240104801688215114304
:108E80000160C1680E4A1140C16001680D4A11407D
:108E900001608168490849008160016801229204EB
:108EA00091430160C168FD2212049143C160002119
:108EB00001610649044888607047000000100240C4
:108EC0000C40FF88F6FFF6FE0050000800ED00E0C1
:108ED00070B501F07BF81D4C1D4D606402E001F09F
:108EE00075F86064A842FAD1207801250526ED03C3
:108EF0003607002804D001280FD0022823D120E013
:108F0000012229463046FDF71EFDFFF7F1FC002245
:108F100029463046FDF717FD15E0607A0122401E14
:108F2000607229463046FDF70EFDFCF733FF002244
:108F300029463046FDF707FD607A002803D12070EE
:108F400001E0FFF7C9F900F033FF70BD48000020D1
:108F50003001CADE10B5818CC90707D001684A68A4
:108F600001235B049A43836A1A434A60818C890710
:108F700007D501684A6801231B049A43C36A1A4350
:108F80004A60818C490707D501684A6801239B0420
:108F90009A43036B1A434A60818C090707D501681D
:108FA0004A680123DB039A43436B1A434A60818C6E
:108FB000C90607D50268916801231B039943836B97
:108FC00019439160818C890607D501688A6801235D
:108FD0005B039A43C36B1A438A60818C490612D59E
:108FE00003685A6801210905046C8A4322435A60C8
:108FF000026C8A4207D10268516803235B059943DA
:10900000436C19435160818C090607D501684A6891
:109010000123DB04806C9A4302434A6010BD0000C8
:10902000F8B500260446C667FDF794FC054620689F
:109030000068124F000709D501212B46002249057F
:109040002046009700F054FA00280DD120680068EF
:1090500040070BD501212B460022890520460097A9
:1090600000F046FA002801D00320F8BD20206067F8
:10907000A067603426740020F8BD0000FFFFFF01E8
:10908000F8B5184CC826E078002829D16079002866
:1090900026D101206071144D686B002700281ED076
:1090A000686BC821081A15E01048E168405C6169E6
:1090B00088470F480A21008848430E490880E06825
:1090C000401CE060E068C82800DBE760696BC820EE
:1090D000401A761EE168814201D0002EE4DC6771FF
:1090E000F8BD00003000002000000240580C0020B5
:1090F000CC000020D600002070B5224CE07800287B
:109100003FD1207900283CD1012020711E4EF16909
:1091100000250906002933DA2156625791420AD107
:10912000F06940062CD5A079002829D0A5712089A6
:10913000401C208124E0A179002903D1A0710A20DC
:1091400000F0D3FC00202056CC2148430F494218A0
:10915000206912181279B262401C00222061A256C6
:10916000CC235A43895881420ADC25612078401C6F
:10917000207020780E2800D12570A078401CA070A7
:10918000257170BD30000020003801403001002002
:1091900010B5806A0022014640314A834A82FEF7B8
:1091A00064FA10BD70B5846A606FA56F2168896824
:1091B00000260906002906DA212804D15220065388
:1091C000204600F047F820688068400606D5222D2A
:1091D00004D15A200653204600F02CF8E06F1021ED
:1091E0000843E0672046FEF740FA70BD10B501461F
:1091F0000968806A0968890614D400225A210A5233
:1092000001680A68FF2301339A430A6001688A688B
:10921000520852008A6001688A6840239A438A6033
:1092200020218167FEF7BCFB10BD10B5806AFEF7F8
:10923000B8FB10BD01680A68FF2321339A430A6016
:1092400001688A68520852008A60202181670021E3
:109250000166704701680A68C0239A430A602021AA
:109260004167704770B5164CE278002A0CD122791C
:10927000002A09D10122E2700025C82903DC02225C
:10928000A256002A01DCE57070BD0123E356CC2212
:1092900053430C4AD1500123E356CC2673439B1809
:1092A0000A460146181DFBF769FF6078401C607094
:1092B00060780E2800D16570A078401EA070E2E7AB
:1092C0003000002030010020F8B504462669A2686D
:1092D000E76932436669102000253E432368324324
:1092E00078491E68784F3E4016431E6023685A68CE
:1092F00003263603B243E66832435A602368A26904
:109300008B4201D0266A32439E680B273F02BE4340
:1093100016439E606D4E23686D4AB3420CD1D268ED
:109320009207920F06D0012A38D0022A34D0032A9D
:1093300020D11EE001201DE0664EB3420AD1D26862
:109340000C26324026D0042A28D0082A24D00C2A01
:1093500010D10EE08B420DD1D66803229202164046
:1093600018D001229202B61A18D0B61A14D096421A
:1093700000D10820564A0126403A574FF6038B4247
:1093800036D100280CD002280DD0042812D008288D
:109390001FD11CE00020EDE70220EBE70420E9E705
:1093A000FDF774FE08E01068C00601D5384605E0F8
:1093B0004A4803E0FDF78AFE002873D06268510036
:1093C0005118814205D81103814202D303E030468F
:1093D000F4E7012566E0010E06025008002330186C
:1093E0005941FBF79BFE03210902411A3C4A55E013
:1093F000E169B14232D1030000F081F909070A0D99
:1094000006250606062B0600E3E7FDF73FFE1CE0F7
:10941000FDF74CFE19E010686168C00602D54808E7
:10942000304A01E0304A48088018FBF761FE80B2FC
:1094300001462E4A10399142CBD8511C01400007F9
:10944000400F08432CE0FDF741FE616840004A08E8
:10945000EAE76168012248081204E5E7030000F02A
:109460004EF909070A0D06260606062C0600B0E787
:10947000FDF70CFE1DE0FDF719FE1AE010686168AB
:10948000C00602D54808C01902E014484A0810185E
:10949000FBF72EFE80B20146144A1039914298D84B
:1094A0002168C8600020206660662846F8BDFDF788
:1094B0000DFE61684A088018EAE76168480880196B
:1094C000E6E7000000480040F369FFEF0038014084
:1094D000401002400044004000093D000024F40018
:1094E000FFFC0F0000127A000048E801EFFF0000C7
:1094F000FFB581B017460E4604460A9D09E0681C78
:1095000007D0FDF727FA0499401AA8420CD8002D7D
:109510000AD02068C1693046884318D00020B8427C
:10952000EDD0002005B0F0BD20680168FF22A13217
:1095300091430160206881684908490081602020CA
:109540006067A0670020603420740320EAE70120F0
:10955000E5E7000010B504491020096808620248D8
:10956000FEF784F810BD00001015002001490D2001
:10957000887070473000002010B507480A22018A21
:1095800051434183FEF75CFDFEF73EFEC8220349CE
:109590000348FEF7A9F910BDBC000020580C0020BC
:1095A00010150020F8B53D4C002321783C4A1D469B
:1095B000082910D0072945D006294ED0052950D0BA
:1095C000042951D0032952D0002954D0012956D062
:1095D000022958D059E0A17800264A1F04E0304FF4
:1095E000BF5DFB189BB2761C9642F8DB6679277943
:1095F0009A195118E3786278C9188918C91940185E
:10960000C0071AD0012E14D0022E16D125482449A5
:10961000C018FBF7B3FD00F0C5FF642000F05EFA50
:10962000BFF34F8F21492048C860BFF34F8F00BF61
:10963000FDE759081046FFF755FB2570E570A5704A
:10964000A571F8BDA1795054491CC8B2A071A17888
:10965000491F8842F5D1082001E060700720207082
:10966000F8BDE0700620FAE760710520F7E7A0700A
:10967000E5700420F3E7552807D10120EFE7AA2879
:1096800003D10220EBE7032803D02570E570A57015
:10969000F8BD032020702071F8BD0000B300002049
:1096A00064130020200D00200400FA0500ED00E006
:1096B0000FB410B503A9044B044A029800F002F954
:1096C00010BC08BC04B0184701A30008F00000203B
:1096D0002021020C01D010211046020A01D01046B0
:1096E0000839020901D01046091F820801D010462E
:1096F000891E420801D0881E7047081A704730B48E
:109700007446641E2578641CAB4200D21D46635D1E
:109710005B00E31830BC184702E008C8121F08C1FC
:10972000002AFAD170477047002001E001C1121FE2
:10973000002AFBD1704708B50021684601706B46CE
:10974000012202212C2000F07BFD022168460170DD
:109750006B4601222C2000F073FD08BD38B504468D
:109760006D20694608706B46012207492E2000F0E3
:1097700067FD0649002C01D0054A00E0054A2E206D
:1097800000F044FD38BD0000060800000618000087
:10979000070600000716000038B504466B46022293
:1097A0000021362000F018FCB3212300FFF7A7FFAB
:1097B0000E0F08153A3A3A3A1C273A3A2F34483AEB
:1097C00000216846017040784108490014E069466C
:1097D000087880088000401C04E06946087880080A
:1097E0008000801C08701DE0684602780A404832FC
:1097F00002704178802001436846417012E068465B
:1098000002780A40027040784106490EF4E7694642
:1098100048780221084303E069464878FD21084062
:10982000694648706B4601220021362000F008FD91
:10983000012200AB11463620013300F001FD38BD96
:1098400069460878CF21084069462030CAE708B544
:10985000032168464170012101706B4602220021FC
:10986000362000F0EDFC0122D20306212D2000F06D
:10987000CDFC012000F032F90120FFF78DFF08BD7B
:1098800008B5020A69464A7008706B460222042134
:109890002D2000F0D5FC0320694608706B4601229C
:1098A00006212D2000F0CCFC0020694608706B4694
:1098B000012206212D2000F0C3FC0A212D2000F0FA
:1098C00071FB08BDFFB58DB00446002506E02528D4
:1098D0000AD0109A0F999047641C6D1C20780028BC
:1098E000F5D1284611B0F0BD00270121484A009764
:1098F00000E00743641C23780846203B9840104250
:10990000F7D120782E2817D1042007436078641CF3
:109910002A280CD10E98641C02C800910E900BE00E
:1099200000990A22514330394018641C0090207875
:10993000014630390929F3D920780028D1D064288C
:1099400008D0692806D075281ED0109A0F99904724
:109950006D1C5BE00A200E99019001C90E91002850
:1099600002DA40422D2102E0390504D52B216A4656
:109970001172012103E0F90704D02021F7E70BAEB3
:109980000B910DE00021FAE70A200E99019001C920
:109990000E91F7E70199FBF7ABFB3031761E317082
:1099A0000028F7D103A8801B20300190780701D54B
:1099B000009801E0012000900199884201DD401AE1
:1099C00000E000200027009006E002A8109AC05D89
:1099D0000F9990476D1C7F1C0B988742F5DB04E0C4
:1099E000109A30200F9990476D1C0099481E0090E6
:1099F0000029F5DC05E03078109A761C0F99904725
:109A00006D1C0199481E01900029F4DC641C65E777
:109A100009280100F8B54A002B4B520DD6182B4AE5
:109A20000C460546142E2BDA002E12DA284BFBF7D3
:109A30006DFC00221346FBF793FF40D2002C03DAA3
:109A40000124E40700253AE02046284337D0214C82
:109A500014E0214F0B46F7403B402B4331D01C4BC9
:109A6000FBF754FC00221346FBF77AFF27D2002CA9
:109A700003DD01200005F0400419BC4300251EE071
:109A8000332E1EDC33460027143BFF43DF403842B1
:109A900017D00F4BFBF7E4FC00221346FBF760FFE7
:109AA0000DD2002C0ADD142E0CD03420811B012095
:109AB00088404019A84200D2641C0546BD43214697
:109AC0002846F8BD641CF9E701FCFFFF9C7500887F
:109AD0003CE4377E0000F03FFFFF0F007D2110B512
:109AE000C900484300F001F810BD002140E000BF6C
:109AF00000BF00BF00BF00BF00BF00BF00BF00BF6E
:109B000000BF00BF00BF00BF00BF00BF00BF00BF5D
:109B100000BF00BF00BF00BF00BF00BF00BF00BF4D
:109B200000BF00BF00BF00BF00BF00BF00BF00BF3D
:109B300000BF00BF00BF00BF00BF00BF00BF00BF2D
:109B400000BF00BF00BF00BF00BF00BF00BF00BF1D
:109B500000BF00BF00BF00BF00BF00BF00BF00BF0D
:109B600000BF00BF00BF00BF00BF00BF00BF491C57
:109B70008142BCD370470000FEB50446002001902E
:109B800000906079734940000E5A61782578491E2B
:109B90007148CFB20163042D77D0072D75D0002115
:109BA0000291217801736C49E37901229205896958
:109BB000002B6CD0914381616748217A4173217AEF
:109BC00082698907890B0A4382610021042000F021
:109BD00028FB324661492E2000F018FB3846FFF77B
:109BE000BDFD5F4E0522705D810040185D49431840
:109BF00007212B2000F024FB5B49029801220B185F
:109C00000B21282000F01CFB705D584980000A5889
:109C10000C21282000F005FBE07955498000401810
:109C2000A1794900425A0221272000F0EFFA514859
:109C30007E00825B0421272000F0E8FAE07900280A
:109C400029D0A07804282CD0282069460872202228
:109C50000621272000F0DAFA02AB01222621272074
:109C600000F0EEFA444938014018E1788900425882
:109C70000821272000F0D5FAA17A601C627A090237
:109C8000114313D016E000E001E0012188E7114301
:109C9000F608816190E764220621272000F0B6FAD9
:109CA000E0E71020694608720246D1E733490172A5
:109CB000090A4172417A007A0A02024320212720D0
:109CC00000F0A4FA2E4F0C2123203A6800F0A9FAE4
:109CD000F01982880421232000F098FAA079002846
:109CE0000BD0E0792749012243180021212000F000
:109CF000A7FA03200190012000902A07120F1001FB
:109D00000243607800218007000B024301980005A0
:109D100002430098400402432079C00640090243F0
:109D20006079C00602431F2000F07BFAA0786178BA
:109D30000123084302040848DB030261E179490377
:109D400019430A4302610021082000F06AFA00204A
:109D5000FEBD000070A60008F400002004280000EA
:109D600018A60008010000201F00002020A60008FF
:109D700040A600084CA6000850A6000841100000AC
:109D800038A600082100002038B50C4607498A8B08
:109D9000002102432C2000F039FA684604706B461B
:109DA000012206212C2000F04BFA38BDF4000020DF
:109DB00010B5FFF7C0FC10BD10B5044604213620D5
:109DC00000F0F0F80121C902002C01D0084300E0A6
:109DD000884302460421362000F023FA10BD00001B
:109DE00038B540206946087000210E2000F0DAF8EE
:109DF0000446002211460E2000F013FA6B460122A1
:109E000000210D2000F01CFA074A00210F2000F06D
:109E100008FA00F0E1F9224600210E2000F001FAD4
:109E200002480021017338BDF8FF272414010020E7
:109E30007CB505460420694608704B4C00206075CF
:109E400021462031206348710873A0836063A063BA
:109E500000F0BCF8454E206002E000F0B7F820604A
:109E6000B042FAD10020FFF797FC4148007824283F
:109E700001D9243806E00621FBF73AF90622101A28
:109E800040010843020601040A4301020A43024357
:109E900000211E2000F0C5F96B460122002124207C
:109EA00000F0CEF91E20FFF7EBFC86B2300AA0735B
:109EB0000420FFF7E5FC0006000E0DD002206946E5
:109EC000087101AB012212212D2000F0B9F9A08BFD
:109ED000012109030843A08300F078F820600620E0
:109EE000FFF7CEFC60600720FFF7CAFCA060F00619
:109EF000C00E207501D110202075C0B200F0DCF931
:109F0000E80707D0FFF7A3FCA08B0121C902084393
:109F1000A0830AE00521362000F02EF815490840FC
:109F200002460521362000F071F90120FFF734FCCC
:109F30000021042000F036F8A0610021262000F066
:109F400031F815218903084302460021262000F03C
:109F500068F900222621362000F058F900F036F882
:109F6000206000207CBD0000F40000203001CADE2B
:109F700000000020FFFD000038B5094C89B280B216
:109F80006B46022200F028F8002806D16846407887
:109F9000010268460078081884B2204638BD0000E7
:109FA000FFFF000038B50024E44389B280B26B465D
:109FB000042200F011F8002806D103216846435C12
:109FC0002202D418491EFAD5204638BD10B500210A
:109FD0000846FFF7E7FF10BD38B5002909D0402437
:109FE00020436C462070C8B27F2906D860700220DA
:109FF0000AE069460870012006E0802420436C4690
:10A000006070C809A0700320694600F0A5FA38BD49
:10A0100010B5144603460A4621461120FFF7DCFF1F
:10A0200010BD10B50346052200211520FFF7D4FF0F
:10A0300010BD10B50346052200211720FFF7CCFF05
:10A0400010BD38B5054600206946087000F0C4F818
:10A05000FF2401342246002D01D0032212020021E8
:10A060000D2000F0D3F8002D13D06B460122032100
:10A070000F20FFF7B1FF68460078000709D5FFF70A
:10A08000AFFE224600210D2000F0C0F80020C043A2
:10A0900038BD002038BD10B5024601210A2000F06D
:10A0A000C0F810BD10B5044600211A20FFF77AFF52
:10A0B000000D22030005120B024300211A2000F0BC
:10A0C000B0F810BD10B5024602492E2000F09EF8EF
:10A0D00010BD000004180000F8B505466B460122CB
:10A0E00003210420FFF778FF0126114C3607002DCD
:10A0F0000DD02A4600210C2000F088F86946087827
:10A100001021084369460870A069304307E069469A
:10A110000878EF21084069460870A069B0430B46F3
:10A12000A06101220321042000F08AF8F8BD00009C
:10A13000F400002010B502460021182000F066F857
:10A1400010BD0000F8B50746002568460570B80741
:10A15000204C2E4600280ADA8020694608706B469B
:10A16000012200210D2000F06BF801202073F80778
:10A170006946087821D006210843694608706B4675
:10A18000012200210D2000F05BF803210F20FFF7D2
:10A19000F3FE8121C900084219D0402069460870A9
:10A1A0006B46012200210D2000F04AF80020FFF745
:10A1B00003FE00252673ED4309E0022108436946AA
:10A1C00008706B46012200210D2000F039F8284666
:10A1D000F8BD0000140100201CB56B4601220321CC
:10A1E0000F20FFF7F9FE684600784022C1091040B1
:10A1F000C9014000814208D0012069460871024629
:10A2000001AB03210D2000F01BF81CBD08B56B4607
:10A210001A70120A5A7089B280B2022200F010F845
:10A2200008BD38B500236C46E254120A5B1C042BAF
:10A23000FADB89B280B22346042200F001F838BD6F
:10A2400038B58024002909D0C02528436D462870E0
:10A25000C8B27F2907D86870022009E02043694608
:10A260000870012004E020436870C809A87003202A
:10A27000694600F0ADF938BD10B514460123121837
:10A280009B029A4202D90020C04310BD0B46821E99
:10A2900021460920FFF7D4FF002010BD10B5054A64
:10A2A0008905126901430A4300210820FFF7B9FF1D
:10A2B000002010BDF400002038B504466B46012292
:10A2C0000E212B20FFF788FE68460078E106400942
:10A2D0004001C90E0143684601706B4601220E2100
:10A2E0002B20FFF7ADFF38BD10B5002142541C06EE
:10A2F000120A22431B0A491C0429F7DB10BD000087
:10A3000013B501231A4669460248FDF74BFB009836
:10A310001CBD0000101500207CB5002425466846B1
:10A32000FFF77FFE04206946220E2D02154322020C
:10A330000C5C1443401EF7D5204629467CBD7CB5F5
:10A34000002425466846FFF774FE04206946220E65
:10A350002D02154322020C5C1443401EF7D5204603
:10A3600029467CBDFCF704FBFEF73CFDFDF77CFEB7
:10A3700037493848002522C005608561C5613649E6
:10A380000562C1600838FCF70DFCFDF759FEFDF7CA
:10A390003BFFFDF717FFFDF71FFE052601223607DD
:10A3A000D1033046FCF7CFFAFEF7E4FBFDF718FDCA
:10A3B000FBF7A0FBFBF76EFB0721B015FFF7E4FCF2
:10A3C000264C0A21208A012248436083170339461C
:10A3D0003046FCF7B8FA1F48C82221498830FDF7FB
:10A3E00083FA204EE07800282FD0FEF7FBFCE570C2
:10A3F000FBF796FD20700F2809D901223946304617
:10A40000FCF7A1FAFEF764FD0022394609E00122BB
:10A4100051033046FCF797FAFEF75AFD002201215E
:10A4200049033046FCF78FFAFDF71EFC608B0028CD
:10A4300001D0401E60830C48618B00780843D1D165
:10A4400001210846FCF7A0FCCCE7FDF70DFCC9E7AD
:10A45000007C004088140020FFFF0000BC000020AA
:10A46000580C0020000400503600002010B586B0C3
:10A470001748FCF71CFB14216846FAF798FE1548AC
:10A4800000900320019000200290052069460007FB
:10A49000FCF794F969461048FCF790F969460F48B3
:10A4A000FCF78CF901210846FCF76EFCFF2401340F
:10A4B0002046FCF741FC0A49086804221043086062
:10A4C0002046FCF749FCFCF74FFC06B010BD00002D
:10A4D00088140020FFFF0000000400500008005016
:10A4E0000070004010B50122920218491848FBF78D
:10A4F00077FB1648174902888A4225D0018004213B
:10A500008180FF21F531C1800A21018100211E22B5
:10A510004181D24382810122C28101840182418230
:10A520008182C182018381834323C38602230387FF
:10A53000782343878287C287024640321184518440
:10A540009184C18300F02EF810BD0000200D002082
:10A5500000FC0008AA550000F0B58C460025102626
:10A56000052109078E620E4C08E067467F5DE760B3
:10A57000A768FF07FCD0E7681F706D1C8542F4DBFD
:10A580000020074606E0E760A568ED07FCD0E56817
:10A590001D54401C9042F6D38E610020F0BD000097
:10A5A0000030014070B572B60124074DA402214667
:10A5B0002846FBF7FBFA002804D022460349284628
:10A5C000FBF798FB62B670BD00FC0008200D002070
:10A5D000F0B50025102605279C463F070B46BE62B6
:10A5E0000C4C06E0595DE160A168C907FCD0E16848
:10A5F0006D1C8542F6DB002007E06146095CE160E6
:10A60000A168C907FCD0E168401C9042F5D3BE6147
:10A610000020F0BD003001400000010203040005ED
:10A62000405C0000A05C0400C06C0800805C04007A
:10A63000E03F1E00E07D1E0007A9022570889B8870
:10A640000A001600010006000100020087008D00CC
:10A650002D001A3152001A339A001A351D011A378B
:10A660006B003B31BE003B335E013B3596023B370E
:10A67000000099599959EB518F421E45142E0080C4
:10A68000EB51F5283333E13A703DE13AC235852B81
:10A69000C2353333C235C235AE47E13A5138A33003
:10A6A000513800000000000000000102030406070A
:10A6B0000809030406080C101820300000000001EF
:10A6C00002030400E4A6000800000020F4000000DB
:10A6D00018970008D8A70008F400002044190000CB
:10A6E0002897000800070400091E080540082609ED
:10A6F0001040085608054008261D040008BE1D0429
:10A700000008BED8BC401008010000000000C8428C
:10A710000000000000000000000000000000000039
:10A720000000000000000000000000000000000029
:10A730000000000000000000000000000000000019
:10A740008C0A000000000000000000000000000073
:10A7500000000000000000000000000000000000F9
:10A7600000000000000000000000000000000000E9
:10A7700000000000000000000000000000000000D9
:10A7800000000000000000000000000002020400C1
:10A790000909010200810000000000000100000022
:10A7A00000000000000000000000000000000000A9
:10A7B0000000000000000000000000000000000099
:10A7C0000000000000000000000000000000000089
:08A7D000000020000000000061
:04000005080050C1DE
:00000001FF
